:100000000C94F0040C9442050C9442050C944205A7
:100010000C9442050C9442050C9442050C94420544
:100020000C9442050C9442050C945D240C94192404
:100030000C945A250C9442050C9442050C944205EC
:100040000C9442050C9442050C9442050C94420514
:100050000C9442050C9436250C9442050C944205F0
:100060000C9442050C9442050C9442050C944205F4
:100070000C9442050C9442050C9442050C944205E4
:100080000C9442050C9442050C9442050C944205D4
:100090000C9442050C9442050C9442050C944205C4
:1000A0000C9442050C9442050C944205050109800C
:1000B000A101850319012AB700150126B700950192
:1000C00075108100C0050C0901A101850419012AE0
:1000D000A002150126A002950175108100C00660DE
:1000E000FF0961A1010962150026FF00952075082E
:1000F00081020963150026FF00952075089102C052
:1001000005010906A101050719E029E715002501E8
:10011000950875018102950175088101050719008F
:1001200029FF150026FF00950675088100050819AE
:10013000012905950575019102950175039101C08D
:1001400000000000000000000000000000000000AF
:10015000000000000000000000000000000000009F
:10016000000000007E0F00D4FFFFFFC700000078F2
:1001700000000000000000002A2B28000000000002
:100180000000000000000000000000290000000046
:100190002C1E3420212224342627252E362D3738B4
:1001A000271E1F202122232425263333362E3738BD
:1001B0001F0405060708090A0B0C0D0E0F1011127B
:1001C000131415161718191A1B1C1D2F3130232D47
:1001D000350405060708090A0B0C0D0E0F10111245
:1001E000131415161718191A1B1C1D2F3130354CF6
:1001F000FD377A585A000004E6D6B44602002101C1
:1002000016000000742FE5A3E016D103915D003DB8
:100210008889C65436C3174FE4DB9143616BF28F74
:100220001A6A60882079D849F518F2E65ED84F8EB0
:10023000C880B3CB94B1E1C84CE54423B326C2CE09
:1002400073131B2197294A73884C66B6C525F88F0E
:10025000748E05B4E15FE6D9F8C5EB1D9533124CF9
:10026000ED3820FABAF466AB7E27172DE3CD884827
:100270005C6E3C59FAE73FAA452D4A5B72E30B14CA
:10028000903CC82D53AA88EB2B9C8A6DC6B247D6EA
:10029000FD8E1EFA510F38630F1919609EADEA7971
:1002A000952A82368C1B541E7995001E8411B34DFD
:1002B00066E86C7C354035A1AE459CEB564E77D454
:1002C0009F23E10E96DB82F3245DDC85E4BDF725F8
:1002D00000485809AAF804F8117637CE536940153A
:1002E0009E2607C2013D59F31B7D9B70613CC826C9
:1002F000343C9861A92D0F51C9C7EDBB59E9D1CB49
:10030000A803FE5E9C322D0FDB764F10670985B384
:1003100027D66DABC504F554C8FB528634B506CE5E
:10032000398252AA424364A5D0192F23D38F9DC38B
:100330006C295B5E33409068ABD0D114BAD59E9CDB
:10034000135BAF6C86E231AF9C73F541F977094DD1
:100350002DDEC1368B8EBA471BBBE0103B5DDF68DC
:10036000FD5E1C58206205B1D90E5B2756C191660F
:10037000ABAA3A2DC2E3D3D5527FBE0DE0A1DD1169
:10038000463CF3CE46D6DC9D234423CAAA86A8E188
:100390003E02E2558A8CFE7CC1EADD03DB6E659588
:1003A0006DAB0F5C3B17B0FF1D3D13CB3592977BB8
:1003B0006CCE0EC7EE648478A0CF24796F31DF1E37
:1003C000456CE67138A34B2D732D096246D16A1333
:1003D0002857CA42A45E114B972BEA70DAD11DC58B
:1003E00017549F7153038A7B6D583B11457E3E30F5
:1003F000460015D82ED69D7B3A22C5F8BA2232F493
:1004000097588436DD039F51EFF47321A018375CB1
:100410003EF64F92D0646574F0C2F423B76FA23AEF
:10042000DE64D01C1B5610B0AC5B55A57F29F4FAD6
:10043000173330C32A67C33C3861DCCC30C23F5429
:10044000A51E05AC4E54A03E63E72F9F42B64A5A04
:100450003E4B472193D1211A7584AD1C4E2F9DAF81
:10046000AE0B3699467870A40C4EC99CECA1812441
:1004700052CBE5B94B291702BC497F25BFB8784A52
:10048000760E9395DB87D27E748813C0F0E34E001E
:100490001AC92A2DF3B9DCC35AAE72BF09540169D7
:1004A000D018C079FC4E40914EF127CEDD47CDA546
:1004B0006CAFE44ACC01C0C3C1515E8B4E017DEEEE
:1004C000BF3B1EB421F5295E41750635110EF6C8F5
:1004D0003BE8E4A3D6426064CB18A4350E6777915D
:1004E00060A02EC5BE616D6DAF17FA64EB1FCF24FF
:1004F000F7EE1ACE9A1679A2EDCD00EE4C0DD41778
:100500009288A4280E82B1247D925EACE7037C2CF5
:10051000F7CB5EE3A66F01A3E6ED48D2C57BBB76C1
:10052000EB184F0972623926CE4E96580F11F3E937
:100530001B4D3B7AB2431ED570C606B5454E9E2F65
:10054000E3EE2E396D785A395C9D930AD5AFDE847F
:100550009D104A4FEC8E3BAA2F8A1FAA1F69CCAA76
:100560000E3564AE1EE730CCCC7E1603B6ED010B23
:1005700040D5138DC82B747267D6C398A7AACB59E0
:10058000ED5BA3F45566C8381D3E90465047124EA9
:10059000855B2D55A83A40BA81DCBE12A240AC4220
:1005A00000000000B4C7536F48B4F6D70001AD0790
:1005B000D22D00005CAE3F68B1C467FB02000000B2
:1005C0000004595A04001600070009000B000A0035
:1005D0001D001B00060019006400050014001A002D
:1005E000080015001C0017001E001F00200021003D
:1005F000230022002E00260024002D0025002700C5
:100600003000120018002F000C00130028000F000B
:100610000D0034000E0033003100360038001100A8
:10062000100037002B002C0035002A0000002900A4
:10063000E000E300E1008200E20050004F005100C2
:100640005200000000006300000055000000570049
:10065000000053000000000000005400580000009B
:100660005600000000002E00620059005A005B0096
:100670005C005D005E005F00000060006100000043
:10068000000000003E003F0040003C0041004200EE
:100690000000440000004600000047000000430046
:1006A000000045000000480049004A004B004C0093
:1006B0003D004D003B004E003A00E500E600E4003E
:1006C0000000B00001000100010001000100010074
:1006D0000100010001000100010001000100010012
:1006E00001000100010001003A003B003C003D0018
:1006F0003F003E00450042004000440041004300EE
:1007000001000100010001000100010001000100E1
:1007100001000100010001000100010001000100D1
:10072000010001000100010035004C000000010043
:1007300001000100010001000100010001000100B1
:1007400001000000000001000000010000000100A5
:100750000000010000000000000001000100000096
:100760000100000000000100010001000100010083
:100770000100010001000100000001000100000073
:100780000000000001000100010001000100010063
:100790000000010000000100000001000000010055
:1007A0000000010000000100010001000100010043
:1007B0000100010001000100010001000100010031
:1007C0000000010001000100010001000100010022
:1007D0000100010001000100010001000100010011
:1007E0000100010001000100010001000100010001
:1007F00001000100010001000100010001000100F1
:1008000001000100010001000100010001000100E0
:1008100001000100010001000100010001000100D0
:1008200001000100010001000100010000000100C1
:1008300001000100010001000100010001000100B0
:1008400001000000000001000000010000000100A4
:100850000000010000000000000001000100000095
:100860000100000000000100010001000100010082
:100870000100010001000100000001000100000072
:100880000000000001000100010001000100010062
:100890000000010000000100000001000000010054
:1008A0000000010000000100010001000100010042
:1008B0000100010001000100010001000100010030
:1008C00000000100010001006903000002000200B5
:1008D00065030000030001006A0300000400020039
:1008E0004F038107050001006B03000006000200B2
:1008F0005103000007000200670300000800010028
:100900006C030000120002006D03000013000200DF
:100910006F03000009025B00030100A0FA09040054
:10092000000103010100092111010001224000071B
:1009300005810308000A0904010002030000000900
:100940002111010001222200070582032000010776
:10095000050303200001090402000103000000094F
:1009600021110100012232000705840320000A1230
:1009700001000200000008EDFEDB0A010101020394
:10098000011C037600690061006C003A00660036C5
:100990000034006300320062003300630000002E68
:1009A0000341004400420020006B006500790062B2
:1009B000006F00610072006400200063006F006E31
:1009C0000076006500720074006500720000000887
:1009D0000351004D004B0000000403090400BF292F
:1009E00011241FBECFEFDAE0DEBFCDBF04B603FE99
:1009F00027C08091A9039091AA03A091AB03B09165
:100A0000AC038730904BA740B04BD1F41092A903B0
:100A10001092AA031092AB031092AC0314BE84B7D9
:100A2000877F84BF0FB6F894A89580916000886195
:100A300080936000109260000FBEE0E0F8E309953B
:100A400011E0A0E0B1E0EAE5F5E502C005900D9205
:100A5000A037B107D9F723E0A0E7B1E001C01D92AC
:100A6000A93AB207E1F714E0C0EFD4E004C021973F
:100A7000FE010E94F929CF3ED107C9F70E948125C6
:100A80000C94792A0C940000E8EDF0E080818E7FD0
:100A900080831092E2001092DA001092E100A0EE42
:100AA000B0E08C9181608C9380818F77808319BCBA
:100AB000A7EDB0E08C918E7F8C9380818F7E8083B8
:100AC0001092820308952091E4003091E50095E6AC
:100AD000A9012091EC00822F817020FF06C0809137
:100AE000E80080FF06C080E008952091E80022FD24
:100AF0001AC080918F03882389F0853089F0809116
:100B0000EB0085FD0FC02091E4003091E500421715
:100B10005307F9F29150E1F684E0089582E00895D8
:100B200083E0089581E00895EF92FF920F931F9361
:100B3000CF937C018B010E946305C82F811117C0E0
:100B40008091E80085FD0BC08091E8008E7780934E
:100B5000E8000E946305882399F3C82F08C0F701B5
:100B600081917F018093F1000150110949F78C2F89
:100B7000CF911F910F91FF90EF9008958091910375
:100B800087FF13C08091E80082FF06C08091E800D3
:100B90008B778093E80004C080918F038111F2CF9E
:100BA000089580918F038823D9F38091E80080FF16
:100BB000F8CF8091E8008E77ECCF982F9093E900E2
:100BC000242F762F50E0891731F07091EC0020919E
:100BD000ED005091F00021FD07C09F5F973071F745
:100BE0008093E90081E008953091EB003E7F3093DF
:100BF000EB003091ED003D7F3093ED003091EB0044
:100C000031603093EB007093EC002093ED00509333
:100C1000F0002091EE0027FDE0CF80E00895CF9214
:100C2000DF92EF92FF920F931F93CF93DF93C8ED64
:100C3000D0E088818F7E8883E7EDF0E0808181605D
:100C4000808384E082BF81E08093820388818E7FED
:100C5000888302EE10E0F80110821092DA0081EE33
:100C6000C82ED12CF601108288818F7788838881E5
:100C70008068888388818F7D888319BC10928F0358
:100C80001092900310928E0310928D0390EEE92E35
:100C9000F12CF70180818B7F80838881816088833C
:100CA00042E060E080E00E94DD05F60180818E7FF9
:100CB0008083F80180818160808380818860808367
:100CC000F70180818E7F8083888180618883DF91B6
:100CD000CF911F910F91FF90EF90DF90CF900895EB
:100CE000FC01809197039091980386179707A0F0D5
:100CF0006115710529F49091E8009E779093E800C2
:100D000090E06115710551F4911108C08091E800DF
:100D100082FF34C080E00895BC01F2CF80918F0340
:100D20008823C1F18530C1F18091E80083FD30C096
:100D30008091E80082FDEACF8091E80080FFE1CF5A
:100D40008091F3002091F200382F6115710519F0A0
:100D50002830310558F091E02830310509F090E055
:100D60002091E8002E772093E800CBCF81918093EB
:100D7000F100615071092F5F3F4FE7CF80918F03E2
:100D8000882341F0853041F08091E80083FFBECF99
:100D900081E0089582E0089583E00895089508951C
:100DA00080918403089587E797E7909301088093E3
:100DB000000888E19AE00FB6F894A8958093600047
:100DC0000FBE90936000FFCF9C014FB7F8948091C5
:100DD0007B0390917C03A0917D03B0917E034FBF74
:100DE000821B930B08952FB7F89480917B03909109
:100DF0007C03A0917D03B0917E032FBF08952091C5
:100E00007803309179032817390771F090937903AB
:100E100080937803E0917603F0917703309721F087
:100E20000084F185E02D0994089520917403309198
:100E300075032817390771F0909375038093740335
:100E4000E0917603F0917703309721F00680F781E7
:100E5000E02D09940895E0917603F091770330979F
:100E600021F00190F081E02D099480E00895452B58
:100E700039F0682381E06F3F09F080E081700895C8
:100E800081E0FCCFDC0160914B0380914C03962FF5
:100E9000891301C00895292F30E0F901EE0FFF1FDB
:100EA000ED5BFC4F408151814A175B07A1F487E05D
:100EB0008A9FA0018B9F500D1124455F5C4F81E0FC
:100EC000FA0184839613E6CF2F5F3F4F23703327B9
:100ED00020934B0308952F5F3F4F922F9370D8CFED
:100EE0001092A8021092A702EBE0F3E08581811135
:100EF00002C014821682379683E0E334F807B1F714
:100F0000089580914F039091500390931101809325
:100F10001001089580E0089590910A0292FF06C0A2
:100F2000282F28712830F9F4877F846093FF06C04A
:100F3000282F28712831F1F4877E846120910B02DB
:100F400020FF06C0382F38713830D9F4877F816090
:100F500021FF06C0282F28712831D1F4877E8161B6
:100F600094FD877E0895282F24712430F9F68B7F15
:100F70008860DCCF282F2471243101F78B7E8861B3
:100F8000DDCF382F3171313019F78E7F8860E0CF97
:100F9000282F2171213121F78E7E8861E1CFCF93F7
:100FA000DF93EC0182389105A9F1D8F581339105E1
:100FB00009F496C048F58932910509F48AC08A97E8
:100FC00009F495C0C11522E5D20708F0B6C0C115D5
:100FD00031E5D30708F026C1C83ED10508F09CC012
:100FE000C03ED10560F5C83AD10508F087C0C53AC2
:100FF000D10508F0EFC0C130D10509F12097F9F013
:10100000C430D105E0F440C08533910509F45AC0DD
:10101000C997C1F680910A02837089F0C0EED0E0D2
:101020000EC0833E910599F170F4803E910501F167
:10103000823E910539F680910A0282FD21C0CE01DF
:10104000DF91CF910895863E910561F1873E91052C
:1010500071F1843E910509F0B5CF80910B0281FFBB
:10106000EECF80910A02C7EED0E084FD0DC0E7CF3D
:1010700080910A0280FD07C190910B0290FFDFCFA3
:10108000C3EED0E084FFDBCFD0E0C0E0D8CF8091CA
:101090000A0282FDFBC090910B0290FDBFCF84FF3E
:1010A000CECFF2CF80910A0283FDDDCFC8CF8091F1
:1010B0000A0283FDEEC090910B0291FFF0CFC4EEC7
:1010C000D0E0BDCF80910A0285FFB9CFC9E2D0E060
:1010D000B6CF80910A0285FFB2CFC5E3D0E0AFCF93
:1010E00080910A0286FFABCFCAE2D0E0A8CF809100
:1010F0000A0286FFA4CFC1E3D0E0A1CFCF3BD10548
:1011000018F6C85AD0E0CC0FDD1FC05EDE4F099044
:10111000D881C02DD46493CFC11540E5D40708F021
:1011200064C0C11580E4D80708F05CC0CE019A9570
:1011300081159F4108F483CFA7CFC11536E5D307AA
:1011400018F5C11545E5D40708F084C0C11584E53C
:10115000D80708F07AC09C2F969596959E0123702B
:101160003327C115D34508F462C0C1E0D0E002C006
:10117000CC0FDD1F2A95E2F730E2939FC0011124C6
:10118000C82BD92BDA685BCFC1158AE5D80778F46C
:10119000C11599E5D90708F068C0C11528E5D2073F
:1011A00008F472CFDC2FCC27C06FD06A48CFCE01B5
:1011B00090568115904208F067CF8D2F8F710E9455
:1011C0008C0790E0982F882788279F719C012C2BF3
:1011D000E90149C0C55AD0E0C35EDE4FC881D0E006
:1011E000D0642DCFDF70D06A2ACFCE01E4E096958F
:1011F0008795EA95E1F783702C2F26952695237025
:1012000040E2249F90011124382B8C2F8370C1E081
:10121000D0E002C0CC0FDD1F8A95E2F7C22BD32BA2
:10122000DC680DCFDC2FCC27C16FD06A08CFC1E0BE
:10123000D0E002C0CC0FDD1F2A95E2F720E2929F9A
:10124000C0011124C82BD92BEBCFDC2FCC27C46FC6
:10125000D06AF5CE8C2F0E948C07C82FD0E0DC2FEF
:10126000CC27CC27DF71D062EACE8C2F8F700E9402
:101270008C0734E0D695C7953A95E1F7CF709C2F4F
:10128000EC01D069DCCEC9E3D0E0D9CEC2EED0E02B
:10129000D6CEC6EED0E0D3CE80910802882331F0BE
:1012A0001092080210920702109206020895CF933E
:1012B000C82F80910B0282FD0CC0809108028C1710
:1012C00041F00E94F3069093070280930602C093B8
:1012D0000802CF910895809590918202982390936F
:1012E0008202089590918202892B80938202089550
:1012F000109204021092030210920202089580914B
:10130000510390915203892B89F00E94F30620919A
:10131000060230910702AC01421B530B81E0209181
:101320005103309152034217530708F480E0817053
:1013300008958091820290919A03892B90910502E1
:10134000892B8093720180910802882309F1809192
:10135000510390915203892B29F00E947F0981113A
:101360000E944C098091720190910802892B809310
:10137000720120E084E791E0FC013191CF0131114D
:101380002F5FF1E08A379F07B9F721110E944C09BE
:10139000E0917603F0917703309731F00280F3818A
:1013A000E02D82E791E00994089580911201877FF2
:1013B0008093120190919A039D7F90939A0384FFEA
:1013C00006C08F7E8093120182E00E947209809194
:1013D000120185FF06C08F7D8093120180E20E947A
:1013E00072090C94990980910102811110920102F5
:1013F0000895E4E7F1E09191891303C0DF011197AB
:101400001C9291E0EA37F907B1F70895A4E7B1E03B
:10141000EFEF90E02D91821751F0EF3F19F4211179
:1014200001C0E92F9F5F9630A9F7EF3F09F40895B7
:101430000E2E000CFF0BEE58FE4F82830895209174
:1014400000029091BF01291302C080E0089530E0AE
:10145000F90153E0EE0FFF1F5A95E1F7E054FE4FFC
:101460005181561306C05081581303C05281541342
:1014700004C02F5F3F4F2770E6CF81E00895809131
:1014800000029091BF01981301C008958F5F87708B
:10149000FACF9E3F49F1990F990F990FE92FE80F65
:1014A0009E2F9770E695E695E69583E0E89FF0011C
:1014B0001124E957FE4F50E040E080E0219130E0F8
:1014C000092E02C0369527950A94E2F7217033273A
:1014D000042E01C0220F0A94EAF7822B4F5F5F4F60
:1014E0004330510559F7089580E008959E3F69F112
:1014F000990F990F990FE92FE80F8E2F877041E010
:1015000001C0440F8A95EAF7E695E695E69583E0F3
:10151000E89FF0011124E957FE4F30E020E070E031
:101520005191DF011197CB01022E02C0969587954C
:101530000A94E2F7817081958527842385278C930F
:101540002F5F3F4F2330310559F70895E92FE2957A
:10155000EF70E250EE3070F4F0E0E558F54D0C9489
:10156000F929803F19F020F4883E20F481E00895A5
:10157000843FE1F380E00895883EC0F3813FD1F7D6
:10158000F5CF93FB882780F9089590E080E00E94D2
:10159000150790E080E00E94FF0610929A031092D7
:1015A00005020C949909809399030C94C50A8091C3
:1015B0009903982F9670963019F488600C94D30A8A
:1015C000877FFCCF21E030E001C0220F8A95EAF747
:1015D00020958091990382230C94D30A9091040260
:1015E0008095892380930402282F277091F4282F57
:1015F000082E000C330B9217130659F090910B0232
:1016000092FD07C08595859585950E94E20A0C9408
:101610007809089521E030E001C0220F8A95EAF7A9
:1016200080919903822B0C94D30A90910B0292FD26
:1016300010C098E0899F90011124622B60930402EE
:101640000E940A0B0E94F306909303028093020209
:1016500008950C940A0B809309020C94C50A882300
:1016600041F0809590919A03892380939A030C947A
:1016700099090895882339F090919A03982B9093B3
:101680009A030C9499090895882321F00E946B090C
:101690000C9499090895882321F00E9472090C94F2
:1016A00099090895882309F44BC0823871F40E9487
:1016B0002B0781FF45C089E30E94060A0E94990911
:1016C00089E30E94F9090C949909833859F40E941E
:1016D0002B0780FF35C083E50E94060A0E94990906
:1016E00083E5EFCF843859F40E942B0782FF28C08E
:1016F00087E40E94060A0E94990987E4E2CF9CEFE2
:10170000980F913AF0F290E2980F983050F4877069
:1017100091E001C0990F8A95EAF7892F0E946B0921
:10172000D2CF9BE5980F933020F490E080E00C94AA
:101730001507885A873120F490E080E00C94FF066A
:1017400008959C013A9521153F4150F5FC01EE2783
:10175000F170BC0166277270AC01442754709C0183
:101760002227387094FF0EC080E1EF2B09F480E04F
:10177000672B09F08062452B09F08064232B89F0E8
:101780008068089581E0EF2B09F480E0672B09F071
:101790008260452B09F08460232B19F0886008953E
:1017A00080E00895CF93DF93EC010E94520BCE01AD
:1017B0000E94A10B9E01205E31092830310510F0F6
:1017C000CD2B21F4DF91CF910C94440BDF91CF917D
:1017D0000C942F0BE82FE695E695E695EF70F0E078
:1017E000E45FFD4F9081482F477021E030E001C059
:1017F000220F4A95EAF787FF04C02095292320830A
:101800000895292BFCCF80937F037093810360930D
:10181000800380918F038430F9F48093E9008FEF87
:101820009091E800815095FD06C095ED9A95F1F7ED
:1018300000008111F5CF8091E80085FF0DC050E0D8
:1018400040E063E070E08FE793E00E9494058091B0
:10185000E8008E778093E8000895BC0184E00C9442
:10186000030CBC0183E00C94030CCF93DF93EC01D9
:1018700081E08093E9008FEF9091E800815095FD21
:1018800006C095ED9A95F1F700008111F5CF809192
:10189000E80085FF14C050E040E068E070E0CE0151
:1018A0000E9494058091E8008E778093E80088E09C
:1018B000FE01A5E8B3E001900D928A95E1F7DF9172
:1018C000CF910895019708F40895EFE9FFE031976B
:1018D000F1F700C00000F6CFCF93C82F882309F49A
:1018E00084C08238C1F40E942B0781FD7EC089E349
:1018F0000E94060A0E9499092FEF81EE94E0215080
:1019000080409040E1F700C0000089E30E94F9099F
:10191000CF910C9499098338A1F40E942B0780FD84
:1019200064C083E50E94060A0E9499092FEF81EEA8
:1019300094E0215080409040E1F700C0000083E532
:10194000E5CF8438A1F40E942B0782FD4EC087E4C6
:101950000E94060A0E9499092FEF81EE94E021501F
:1019600080409040E1F700C0000087E4CFCF8CEFCB
:101970008C0F813A68F4E4E7F1E08191C81779F1BE
:1019800021E0EA37F207C9F78C2F0E94060AC0CF80
:1019900080E28C0F883048F4C77081E001C0880F66
:1019A000CA95EAF70E947209B3CFEBE5EC0FE3307A
:1019B00040F4F0E0E35EFE4F808190E0CF910C9424
:1019C0001507C85AC73188F4EC2FF0E0EE0FFF1F5F
:1019D000E05EFE4F80819181CF910C94FF068C2FA9
:1019E0000E94F9090E949909CFCFCF910895CF9312
:1019F000DF93EC01662329F080919A038260809343
:101A00009A03CE019056811520E2920720F0905E55
:101A10008115904108F4DD27CE010E94A10B9E01A3
:101A2000205E31092830310510F0209739F40E94EA
:101A30004B0B8C2FDF91CF910C946C0C0E943A0BC6
:101A4000F8CFDF92EF92FF920F931F93CF93DF9324
:101A50007C018B01D42E8091120182FF8CC0C09139
:101A6000A502D091A602CE15DF0521F0E114F10404
:101A700009F081C0809112018B7F8093120181FD5A
:101A800073C08091A3029091A402A801481B590B36
:101A900081E020911001309111014217530708F4A1
:101AA00080E08170F82E80911201F0FA81F9809324
:101AB0001201FE0183E0F695E7958A95E1F7EE7154
:101AC000FF27ED57FD4F20813181AE014F70552723
:101AD00081E090E002C0880F991F4A95E2F7FF204D
:101AE00009F444C0822B932B9183808380918202DE
:101AF00081FF08C08091120180618093120182E011
:101B00000E946B098091820285FF08C080911201BA
:101B100080628093120180E20E946B096F2DCE01DA
:101B20000E94F70CDD2031F080916A0385FF02C02E
:101B300086FF3BC080916D0390916E030E94620C02
:101B40008091A5029091A6029C013056211540E299
:101B5000340720F0305E2115304108F499270E94A7
:101B6000D20B0E94D5091DC081E09BCF8095909536
:101B700082239323B9CFC7019927970130562115A6
:101B800040E2340728F0305E2115304108F0C701EB
:101B90000E94D20B8091A5029091A6028E159F05FE
:101BA00001F31093A4020093A302DF91CF911F9140
:101BB0000F91FF90EF90DF9008951F93CF93DF93E5
:101BC000182FC0916F03D0917003893321F0C09119
:101BD0006D03D0916E03812F0E946C0C209731F41D
:101BE000812FDF91CF911F910C94520B8FE99FE0D1
:101BF0000197F1F700C000002197F0CF0F931F93DA
:101C0000CF93DF93C42FD22FFC0182818823A1F0D0
:101C1000409373030E94F3069093720380937103C1
:101C2000C77081E001C0880FCA95EAF7DF91CF91B4
:101C30001F910F910C944B0B10917303141339C027
:101C400080917103909172030E94E40620916703D2
:101C5000309168038217930760F5C0E2CD0F1D171E
:101C6000B9F080E2810F883040F4177081E001C044
:101C7000880F1A95EAF70E94440BC83048F481E0B7
:101C80009D2F977001C0880F9A95EAF70E944B0B21
:101C9000802F0E94DD0DC83098F4D77081E001C01C
:101CA000880FDA95EAF7DF91CF911F910F910C948D
:101CB000440BC77081E001C0880FCA95EAF7F3CFE3
:101CC000DF91CF911F910F910895AF92BF92CF9264
:101CD000DF92EF92FF920F931F93CF93DF93EC016C
:101CE0008AE0A82E2881222309F48CC02130C9F56E
:101CF00099818A81913021F422960E94DD0D05C0E0
:101D0000923029F422960E946C0C2196EBCF9330EE
:101D100021F422960E94520BF8CF943011F02196B4
:101D2000F4CF229630E020E0AE014F5F5F4F80534A
:101D3000990B8A30910550F02150310930F38FE929
:101D40009FE00197F1F700C00000F6CFA29EB0011E
:101D5000A39E700D11249C01260F371F8981EA0173
:101D6000E3CFE22FF0E0E059FE4FB490822F86954A
:101D70008695869590E0FC01E05AFE4FE49027702E
:101D8000F12C022E02C0F594E7940A94E2F731E0B8
:101D9000E322FF24FC01E05BFE4FC490D12C022E15
:101DA00002C0D594C7940A94E2F731E0C322DD243F
:101DB000FC01E05CFE4F049110E002C01595079510
:101DC0002A95E2F701701127E114F10419F081EE70
:101DD0000E946C0CC114D10419F086EE0E946C0CA8
:101DE0008B2D0E94DD0DCD2819F086EE0E94520B3E
:101DF000EF2819F081EE0E94520B012B09F485CFD8
:101E00008CE27BCFDF91CF911F910F91FF90EF90EC
:101E1000DF90CF90BF90AF900895489906C023E01F
:101E20002A95F1F700000197C1F70895489B06C075
:101E300023E02A95F1F700000197C1F70895509A21
:101E40008AEB8A95F1F700C0509883E091E0019702
:101E5000F1F700C000000895509A83E091E00197E7
:101E6000F1F700C0000050989AEB9A95F1F700C086
:101E70000895EF92FF920F931F93CF93DF93D0E0DB
:101E8000C0E090E8E92EF12C082F10E0C7010C2EDD
:101E900002C0959587950A94E2F780239123892BB8
:101EA00069F00E941F0F2196C830D10579F7DF91A4
:101EB000CF911F910F91FF90EF9008950E942C0FEA
:101EC000F2CFCF93C82FF894509A83EF9BE00197FD
:101ED000F1F700C000000E941F0F8AE20E94390F34
:101EE0000E942C0F8FE193E00197F1F700C00000F2
:101EF0000E941F0F80E00E94390F8C2F87700E9474
:101F0000390F0E942C0F7894CF9108950F931F934F
:101F1000CF93DF930FE413E0C7E2D3E0CE010E943A
:101F20002F2AF80181938F012196C934F3E0DF074E
:101F3000A9F7CAECD8E0FE0185919491009711F0C1
:101F4000FC0109952896F9E0CA31DF07A1F7DF9176
:101F5000CF911F910F9108950F931F93CF93DF930C
:101F6000833030F5603120F5483010F520E1629F74
:101F70008001112450E0440F551F040F151F90E0FD
:101F8000982F8827080F191FC80187960E942F2AAB
:101F9000C82FD0E0DC2FCC27C80188960E942F2ABA
:101FA0009E01282BC901DF91CF911F910F910895B8
:101FB00090E080E0F8CF462F20918002309181029E
:101FC000232B49F4833038F4703128F4683018F446
:101FD000672F0C94AC0F90E080E00895CF92DF92D1
:101FE000FF920F931F93CF93DF936C01009199039E
:101FF00080910902082BC7E0D0E010E0FC2EC80158
:102000000C2E02C0959587950A94E2F780FD0CC0CE
:102010002197A0F7F12C8F2DDF91CF911F910F9178
:10202000FF90DF90CF900895B6018C2F0E94DB0FB8
:102030000E94CF07019761F3EECFCF93DF93EC01BE
:102040000E94EE0FBE010E94DB0FDF91CF910C9436
:10205000CF07FC0186819781009721F00E94CF076E
:102060000C94A60A808191810E941D10F9CF1F93C4
:10207000CF93DF9300D000D00F92CDB7DEB7498366
:102080005A8389819A816623B9F02223A9F00E949C
:10209000EE0F182F682F89819A810E94760A698134
:1020A0007A81812F0F900F900F900F900F90DF91FA
:1020B000CF911F910C94DB0F0E94490A182FEFCF8C
:1020C000FC01262F86819781009739F44081518148
:1020D0006281738184810C943710089583E290E0CB
:1020E0000E942F2A873789F484E290E00E942F2AE9
:1020F0008C3759F485E290E00E942F2A91E08F32CC
:1021000009F090E0892F8170089580E0FCCFCF9393
:1021100084E090E00E942F2AC82F82E290E00E9483
:102120002F2A982F8C2FCF9108950F931F93CF9321
:10213000DF930FE413E0C7E2D3E0CE010E942F2A21
:10214000F80161918F01681719F0CE010E943D2AB4
:102150002196C934F3E0DF0781F7DF91CF911F911A
:102160000F910895EFE4F3E0128E138E8FEA90E062
:102170009183808385E0848F88E893E193838283D1
:1021800082E390E0978B868B88EC90E0918F808F34
:10219000158E8AE090E0978F868F80E590E091A37E
:1021A00080A30E9495100C94860FCF93DF93C9E90A
:1021B000D3E060E0CE010E943D2A2196C11584E063
:1021C000D807B9F7DF91CF9108950F931F93CF935D
:1021D000DF938901833048F5603138F5483028F5C0
:1021E00021153C4531F420910E0130910F01232B34
:1021F000E1F090E1699FE001112450E0440F551F88
:10220000C40FD51F90E0982F8827C80FD91F612FC2
:10221000CE0187960E943D2A602FCE018896DF91DD
:10222000CF911F910F910C943D2ADF91CF911F9177
:102230000F910895CF93C82F6FEF811167E783E265
:1022400090E00E943D2A6FEFC1116CE784E290E0BC
:102250000E943D2A6FEFC1116FE285E290E0CF91BD
:102260000C943D2ACF93C0910B02C2FB992790F9A1
:10227000981799F080FBC2F9C0930B0260910A0293
:1022800084E090E00E943D2A6C2F82E290E00E9460
:102290003D2A82E0CF910C94EE0ACF9108957F926F
:1022A0008F929F92AF92BF92CF92DF92EF92FF9266
:1022B0000F931F93CF93DF93CDB7DEB72A970FB657
:1022C000F894DEBF0FBECDBFA0900E01B0900F01FD
:1022D00081E090E090930F0180930E0184ECC82E72
:1022E00085E0D82E00E0760110E015C0F4012591BC
:1022F0003491472D612F802F0E94E51082E0880ED7
:10230000911C739498E07912F1CFE0E1EE0EF11C8C
:102310001F5F103119F04701712CE8CF0F5FD39484
:10232000033009F70E94B210CE0101967C018AE0C9
:10233000F70111928A95E9F709E413E04AE050E0C9
:10234000B801C7010E94612A065F1F4F0939F3E0F7
:102350001F07A1F7B0920F01A0920E012A960FB6A7
:10236000F894DEBF0FBECDBFDF91CF911F910F91CB
:10237000FF90EF90DF90CF90BF90AF909F908F90A5
:102380007F90089580E00E941A1160E086E290E05C
:102390000E943D2A0E944F110E94D51081E00C94AA
:1023A0001A1110928202E4E7F1E086E0DF011D924B
:1023B0008A95E9F70C94C50A1F93CF93DF93CDB7A5
:1023C000DEB7AA970FB6F894DEBF0FBECDBF81E986
:1023D00093E02091F100DC012D93CD01B3E0893928
:1023E0009B07B9F780919203833009F472C0B8F467
:1023F000813009F449C0823009F4B3C08091E8000B
:1024000083FF96C280919103909192039A3008F0D5
:102410008FC2E92FF0E0E757F54D0C94F9298A3087
:1024200009F48EC08B3009F471C0893039F780917E
:102430009103813219F7809195039091960300974B
:1024400011F00297D9F68091E800877F8093E80029
:102450008091E80082FF38C09091F3008091F200F3
:10246000029731F48091F100813011F0863021F42F
:102470008091F100809384038091E8008B778093B2
:10248000E8000E94BE05BACF80919103813A09F01D
:10249000B5CF8091E800877F8093E8008091950315
:1024A00090919603892B61F468E085E893E070E0F1
:1024B0000E9470068091E8008B778093E8009ECFA1
:1024C00060E090E080E0F3CF80918F038111C0CF76
:1024D00095CF80919103813A09F090CF8091950337
:1024E00090919603892B09F089CF8091E800877F2E
:1024F0008093E8008091E80080FFFCCF8091140178
:102500008093F1008091E8008E77B9CF809191039C
:10251000813209F073CF8091950390919603892BB6
:1025200009F06CCF8091E800877F8093E8000E94DB
:10253000BE0580919303809314010E94D1115ECF58
:1025400080919103813209F059CF8091E800877F13
:102550008093E8000E94BE058091940380938303DA
:102560004DCF80919103813A09F048CF8091E800E6
:10257000877F8093E8008091E80080FFFCCF809106
:102580008303BECF803899F0823809F0D1C18091A1
:1025900095038F70873008F0CBC18093E90080915C
:1025A000EB0085FB882780F91092E90006C0809136
:1025B0008D0390918E03911182609091E800977F36
:1025C0009093E8008093F1001092F1008091E80070
:1025D0008E77AAC1882309F498C1823009F0A8C176
:1025E0008091930381119BC1809195038F702FEF90
:1025F000280F263008F09CC18093E9002091EB0061
:1026000020FF8DC1933031F48091EB008062809384
:10261000EB0085C19091EB0090619093EB0021E07D
:1026200030E001C0220F8A95EAF72093EA00109269
:10263000EA008091EB008860EACF811179C11091A6
:1026400093031F778091E3008078812B8093E300D0
:102650008091E800877F8093E8000E94BE0580910A
:10266000E80080FFFCCF8091E30080688093E30066
:1026700082E0111183E080938F035AC18058823029
:1026800008F056C120919303309194032C3DE3E070
:102690003E07A1F583E08A838AE289834FB7F894E5
:1026A000DE01139620E03EE051E2E32FF0E050938C
:1026B0005700E49120FF03C0E295EF703F5FEF7099
:1026C0008E2F90E0EA30C0F0C7968D939D932F5FD8
:1026D000243159F74FBF8091E800877F8093E8004D
:1026E0006AE270E0CE0101960E9470068091E800D7
:1026F0008B778093E8001CC1C096E7CF809195034B
:1027000090919603432F55274330510509F44AC051
:1027100078F54130510509F485C08BE590E0E4E19E
:10272000F9E04230510509F003C12091E800277F0C
:102730002093E80020919703309198038217930724
:1027400008F49C0140E02115310509F070C04111E9
:102750006EC08091E80082FDC9CF80918F038823ED
:1027600029F2853019F28091E80083FFF2CFBECFC5
:102770004132510509F447C04232510509F0D8C031
:102780008330910508F0D4C0FC01EE0FFF1FEF5A13
:10279000FE4F0190F081E02D825B9E4FDC018C9119
:1027A00090E01DC0332721303105E9F021153105B6
:1027B00079F022303105F9F02330310509F0B8C045
:1027C000E1E8F9E0E4918E2F90E0E1E8F9E007C05C
:1027D000E9EDF9E0E4918E2F90E0E9EDF9E0009762
:1027E00009F4A6C0A2CFEFECF9E0E4918E2F90E0BF
:1027F000EFECF9E0F4CFEFE9F9E0E4918E2F90E00F
:10280000EFE9F9E0ECCF8330910508F091C0880F33
:10281000991FFC01E95AFE4F0190F081E02D89E0FB
:1028200090E083CF82E190E0EFE6F9E07ECF809107
:102830008F03882309F45ACF853009F457CF80914C
:10284000E80083FD53CF8091E80082FD82CF809124
:10285000E80080FF78CF9091F3008091F20021157D
:10286000310519F08830910550F041E0089709F0E2
:1028700040E08091E8008E778093E80064CF449137
:102880004093F1003196215031090196E8CF80380C
:1028900009F04EC08091E800877F8093E800809126
:1028A00090038093F10092CE811142C01091930366
:1028B0001230F0F58091E800877F8093E800109354
:1028C00090030E94BE05112311F084E005C08091A1
:1028D000E30087FDFACF81E080938F0342E061EC53
:1028E00081E00E94DD0542E261EC84E00E94DD05AA
:1028F00042E261EC82E00E94DD0542E260EC83E0AE
:102900000E94DD0580918F0313C080919303813075
:1029100079F481E0933009F080E080938E03109287
:10292000E9008091E800877F8093E8000E94BE055F
:102930008091E80083FF0AC08091E800877F809340
:10294000E8008091EB0080628093EB00AA960FB6BE
:10295000F894DEBF0FBECDBFDF91CF911F910895D8
:10296000CF92DF92EF92FF920F931F93CF93DF935B
:10297000CDB7DEB72A970FB6F894DEBF0FBECDBF36
:10298000E0E3F2E080E5DF011D928A95E9F7EBE0F4
:10299000F3E088E3DF011D928A95E9F780E3C82E12
:1029A00082E0D82E7F0109E413E0F701D182C082D2
:1029B0004AE050E0B801CE0101960E941F2A88E04B
:1029C000FE013196D60101900D928A95E1F7898535
:1029D0009A85D70113969C938E931297BAE0CB0EEB
:1029E000D11CE7E0EE0EF11C065F1F4F0939F3E042
:1029F0001F07D9F62A960FB6F894DEBF0FBECDBFDB
:102A0000DF91CF911F910F91FF90EF90DF90CF90CA
:102A100008956AEE7EEF90E080E00E945B2A60E01D
:102A200082E090E00E943D2A60E083E090E00E9416
:102A30003D2A1092090260E084E090E00E943D2A65
:102A400060E082E290E00E943D2A60E085E090E054
:102A50000E943D2A60E086E090E00E943D2A6FEFF0
:102A600087E090E00E943D2A40E050E0BA0188E013
:102A700090E00E944F2A60E08DE090E00E943D2AA5
:102A800040E050E0BA0188E190E00E944F2A60E007
:102A900087E190E00E943D2A40E050E0BA018CE1DD
:102AA00090E00E944F2A70E060E080E290E00E9497
:102AB0005B2A40E050E0BA0188E190E00E944F2A92
:102AC00080E00E941A110E94C21140E050E0BA0159
:102AD0008FE090E00E944F2A40E050E0BA0183E18D
:102AE00090E00C944F2A8F929F92AF92BF92CF9218
:102AF000DF92EF92FF920F931F93CF93DF9300D05B
:102B000000D0CDB7DEB77C01FC01438154816181E7
:102B100080810E94370781112AC061E0C7010E94AD
:102B200060108C01F7018281882309F46FC6C80107
:102B300082519F45409708F004C68FEF93E00E94B2
:102B40002F2A5EEED52ED00E09E913E0882361F11D
:102B500080910402877059F0F7018281882339F04F
:102B600080910B0282FD03C082E00E94EE0A0F906A
:102B70000F900F900F90DF91CF911F910F91FF90C9
:102B8000EF90DF90CF90BF90AF909F908F9008957F
:102B90000115F4E01F07E1F2C8010E942F2A8111FC
:102BA00001C0DA940F5F1F4FD110F2CF19821A8241
:102BB0001B821C82CC24CA9448012FEF821A920AED
:102BC000C8010E942F2A89831A82882309F4C0CF62
:102BD000813009F048C0580132E0A30EB11CC40195
:102BE0000E942F2A982E8A83882309F4B1CFC50129
:102BF0000E942F2AD82E8FEF890D833068F4580158
:102C000043E0A40EB11CDB82DD2021F0CE01019651
:102C10000E94650E8501D0CF54E09512FBCF58017C
:102C200084E0A80EB11CC80103960E942F2ADD2063
:102C300009F48ECF882309F48BCF8150990BC89E5D
:102C40009001C99E300D1124ED2DE150FF0BCF01F5
:102C5000820F931F0197F0F2EFE9FFE03197F1F750
:102C600000C00000F7CFCE0101960E94650E54010E
:102C7000D1CF81E00E940A0B0E94D70A69CF81E080
:102C80000E94E20AF9CF82E0F5CF809112018160C3
:102C9000809312018DC5809112018E7F8093120165
:102CA0000E94D50985C5809112018F7E013E1105D4
:102CB00031F0053E1105C1F4809112018F7D8093A2
:102CC00012018091120180FF82C5F70182810832D2
:102CD000110528F50E31110508F074C004301105F6
:102CE00080F5811170C573C5C80190568115E0E269
:102CF0009E0720F0905E8115904118F78091120197
:102D000082FF65C580916C0381FD61C52CE731E0D0
:102D100040E0B60190E080E00E94210D58C50933E3
:102D2000110558F40D32110518F40B321105C9F6CE
:102D300090916A0392FDD5CF08C004361105C1F306
:102D4000D0CF90916A0394FDCCCF882309F4A1C021
:102D50009091820280910802282F292B322F3D7FEB
:102D6000B1F11092A6021092A50230916A0331FDD2
:102D70002EC0F80143E0F695E7954A95E1F7EE712C
:102D8000FF27ED57FD4F98012F70332781E090E02A
:102D900002C0880F991F2A95E2F7809590952081AF
:102DA0003181822393239183808360E0C8010E9454
:102DB000F70C809108028D7F0E94570982E00E94E3
:102DC000EE0AC6CE90916A0393FD8BCFBECF38E05A
:102DD000F701ACE7B1E001900D923A95E1F710925E
:102DE0007E011092800110927F01A090A502B09008
:102DF000A6020A151B05B1F530916A0335FF32C0F2
:102E00004091120141FB992490F841FF02C036FF26
:102E100029C04091A3025091A402B601641B750B16
:102E2000409167035091680364177507D8F491FFC8
:102E300008C08091120180618093120182E00E949B
:102E40006B098091820285FF08C080911201806227
:102E50008093120180E20E946B09692DC5010E94D6
:102E6000F70C76CE9091120121FB91F9909312010B
:102E70008D7F0E9457091093A6020093A502D0925D
:102E8000A402C092A3028091120184608093120177
:102E900095CF970140E0B601C8010E94210D58CEA0
:102EA000053F8CE5180709F466C008F45EC0063FCC
:102EB000ECE51E0709F465C0F7013281332309F4FC
:102EC000B1C4109273030330FDE51F0708F065C01D
:102ED0000A3F2CE5120730F4C80182509C45449704
:102EE00008F060C00E94871090930B0280930A0242
:102EF00000315CE5150709F45FC108F0DBC008305C
:102F00009CE5190709F44AC108F0AAC00430FCE5A1
:102F10001F0709F431C108F095C002303CE51307E2
:102F200009F424C180910A02826003301C4509F42F
:102F300020C160910A0210910B0284E090E00E948F
:102F40003D2A612F82E290E00E943D2A0E94D11129
:102F5000FFCD07E225EE45EE68ED7CE553C406E2C1
:102F600021EE40EE63EF7CE54DC407E225EE44EE32
:102F700064EF7CE547C406E221EE42EE65EF7CE5B6
:102F800041C407E225EE46EE66EF7CE53BC408E26D
:102F900021E045EE69ED7CE535C401364DE51407C9
:102FA00009F4A0CF06318CE5180709F43FC40A35AF
:102FB0005DE5150709F451C108F02DC101159CE527
:102FC000190709F43AC10E3D1C4509F443C1F70144
:102FD00086819781009709F444C10E94CF07182F7A
:102FE000092FF701C280D580D2943FE0D32280918F
:102FF00004028770C1F0AC2CCC20B1F0892F807F07
:10300000803421F080E2810F883068F080910B02DB
:1030100082FD09C082E00E94EE0A8091040287705E
:10302000AA24A3948111A12C902E92942FE0922295
:10303000FBE0F91508F49EC1E92DF0E0ED56F54DE1
:103040000C94F92980910A02806106305CE515072D
:1030500009F48FC008F494C080910A02806289C08C
:1030600080910A028D7F0C309CE5190709F481C01C
:1030700070F480910A028C600A30FCE51F0709F4A5
:1030800078C008F48FC080910A028E7F72C0809150
:103090000A02877F0E303CE5130709F46AC080916D
:1030A0000A028B7F0F301C4508F463C080910A022E
:1030B0008F7E5FC00C3F5CE5150709F479C068F5A9
:1030C00004319CE5190709F48BC080F40231FCE55A
:1030D0001F0709F475C080910A028F7B03311C45DC
:1030E00008F447C080910A02837F43C00A3F3CE551
:1030F000130709F449C008F04DC005311C4509F01B
:1031000018CF80910A0282FB992790F921E092273B
:1031100090FB82F990FB83F92CC001158DE518070F
:1031200009F454C088F480910B0283600E3FECE5F3
:103130001E0769F180910B028D7F0F3F1C4538F10E
:1031400080910B028C7F23C002302DE5120709F419
:1031500056C008F44EC001361D4509F0EACE9091E4
:103160000A02892F8F7E94FF806103C080910A023A
:10317000816080930A02DDCE80910A028460F9CFDB
:1031800080910A028860F5CF80910B028160809364
:103190000B02CFCE80910B028260F9CF80910A02A0
:1031A0008064E7CF0E94D11180910A028068E1CF4C
:1031B00080910B028E7FEBCF80910A028F7DD9CF59
:1031C0000E94D11180910A028F77D3CF80910B0298
:1031D000982F909591708E7F892B90FB81F9D7CF96
:1031E0000E94D11190910A02892F97FB87F980588C
:1031F000C0CF61E08EE090E00E943D2A9ACE60E070
:10320000F9CF80918401811104C089E20E94F909FB
:1032100038C385E3FBCF0B35FDE51F0701F10C3506
:103220001D4509F0D4CE80910B0282FB882780F9DE
:1032300091E089270E943211CACE0E94D1113FEF3E
:1032400044E35CE0315040405040E1F700C00000F2
:103250000E94D3060E9409157BCC81E0EBCF80E071
:10326000E9CF828100811181882369F0C8010E9421
:10327000EE0FD82E682FC8010E94760AB8018D2D56
:103280000E94DB0FAACEC8010E94490AD82EF6CFB1
:10329000202F2F70B22E802F807F19F0B29490EFE4
:1032A000B922CC20A9F0BB2059F080E2810F8830F0
:1032B00010F0111107C08B2D0E9472090E9499090C
:1032C000812F56C080919A03B82AB0929A03F6CF04
:1032D000812F0E94520BBB2009F44CC080E2810F69
:1032E000883010F0111104C08B2D0E946B0906C0AC
:1032F000B09480919A03B822B0929A030E949909DF
:1033000039C0302F3F70B32E802F807F803219F06C
:10331000B29480EFB8221123E9F0113009F49FC074
:10332000CC2009F4A8C0DD2009F478C020E0F70122
:10333000408151816281738184810E943710809124
:103340006C0381FDBDCFF701858180FFB9CF8F7000
:10335000858364C080910B0282FF42C0CC20D1F1F2
:10336000BB2029F08B2D0E9472090E94990980E0F0
:103370000E946C0CE92DE850FF0B349728F40E9452
:103380002B0780950E94610F812F902F0E94A60A23
:103390008111B8C11092860110928501AA20A9F06E
:1033A0008091040280FD11C0F701128285958595F8
:1033B00085950E940A0BC7010E9473158091040233
:1033C0008595859585950E94E20A60E0C7010E9477
:1033D0006010CDCB80E00E94520BBB2059F284CF0D
:1033E000CC2001F1D11004C0809108028B2917C0B4
:1033F00041E0D41206C0809108028B290E9457092F
:10340000B9CF80916B03823078F3D812EDCF0E9450
:103410004C0980910102B812B09201028B2D0E94DA
:103420004B0BA8CFD11006C00E944C098B2D0E94D7
:10343000440BA0CF80916B0351E0D5120BC08230BA
:1034400008F498CF809182028B2109F493CF0E94D7
:10345000F309EACF823040F3D812E6CF8BCFCC20ED
:1034600029F085E08D1508F485CFD8CF94E09D151F
:1034700008F480CFDBCFDD20C9F280916F039091FB
:103480007003193321F080916D0390916E030E94B7
:10349000620C812F0E94520B6DCF802F86958695EE
:1034A000837069F0813009F065CF812F902F937080
:1034B000C11002C090E080E00E94FF065BCF812F28
:1034C000902F9370C11002C090E080E00E94150719
:1034D00051CF802F837091F5C1104CCF412F429571
:1034E00046954770440F440F812F8F70042E01C002
:1034F000880F0A94EAF7212F207114FF07C02FE0EC
:1035000030E001C0220F4A95EAF72095302F36951A
:1035100036953370323069F050F440910902313001
:1035200029F0822B84230E942B0B24CF842B822B07
:10353000FACF282B809109028227F5CF8695CC20DF
:1035400011F0802F8170882309F414CF412F429508
:1035500046954770440F440F812F8F70042E01C091
:10356000880F0A94EAF7212F207114FF07C02FE07B
:1035700030E001C0220F4A95EAF72095302F3695AA
:1035800036953370323069F050F440919903313000
:1035900029F0822B84230E94D30AECCE842B822B29
:1035A000FACF282B809199038227F5CFF02FFF7057
:1035B000BF2ECC2029F08F2F0E940A0B812F2FCFF6
:1035C000812F0E94440B8B2D0E94E20AD3CE123F22
:1035D00089F160F4103FB9F0113F81F0CC2009F47B
:1035E0008CC0D1106DCE802F8F7128C0133F49F150
:1035F000143FA1F780910B0282FF2FC0802F8F71A3
:10360000CC2011F31BC0CC2081F024E02D1508F450
:10361000B1CE202F2F7181E090E001C0880F2A9554
:10362000EAF7909199038927B6CF35E03D1508F464
:10363000A1CEEFCF802F8F71C110C6CF0E940A0B91
:1036400099CE80E0CC2009F4A6CF81E0902F9F7125
:1036500001C0880F9A95EAF79ECF80916B03823064
:10366000A0F180910102CC20F1F00E946B098091C1
:1036700004028770843041F40E947809802F8F7192
:103680000E94E20AA12C76CE80916B03D816D0F767
:10369000402F4F71B42E842F0E940A0B63E08B2DB4
:1036A0000E94150BEFCF0E94720980916B03D81610
:1036B00040F00E9478090E94F30964E0802F8F7126
:1036C000EFCF81E00E94EE0ADDCFCC2059F0502FE1
:1036D0005F71B52E852F0E940A0B63E08B2D0E942F
:1036E000150B48CE81E00E94EE0A81E08D1508F0AE
:1036F00041CE82E00E94EE0A3DCED110BECE802F98
:103700008F7162CFCC2019F0D11044CE47CED110AA
:1037100041CE20E0F7014081518162817381848133
:103720000E94371080916C0383FF34CE8091850115
:1037300090918601029709F02DCE812F0E94DD0D18
:1037400029CE0031FFE51F0709F493CA01312FE5A7
:10375000120709F498CA80916A0380FF38C00E945A
:10376000F3066C01F7018281882309F49CCA8091D9
:10377000120182FF08C02CE731E040E0B60190E082
:1037800080E00E94210D0B31FCE51F0709F47DCA82
:103790000C312CE5120709F47ECA90911201892F91
:1037A0008E7F90FF81600A313CE5130709F476CAE9
:1037B000C8019056811540E2940728F0905E81156B
:1037C000904108F07ECA1092A6021092A502033F13
:1037D000FCE51F0709F4C3CB08F062CB083D3CE5CC
:1037E000130709F4B6CB093D4CE5140709F4CFCB18
:1037F000073D5CE5150709F05FCB06E221EE41EEDF
:1038000067ED7CE5C7010E94FE0DA2C900313FE5CE
:10381000130709F434CA01314FE5140709F09BCFAF
:1038200082E02ECA06311C4509F0D1CB809182027C
:10383000982F9A7A2091690320FF04C0482F44747E
:1038400009F090E021FF04C0482F417109F090E099
:1038500022FF04C0482F487809F090E023FF03C0FE
:10386000827209F090E0332309F4CBCC81E091110E
:1038700001C080E08093840189E2911185E30E9478
:10388000060A0E94990964C9CF92DF92EF92FF92D3
:103890000F931F93CF93DF938091BC01807F31F40E
:1038A0008091B901C091000281110BC0DF91CF91CD
:1038B0001F910F91FF90EF90DF90CF900895219688
:1038C000C7708091BF018C1789F3F090B701E09029
:1038D000B801C090BA01D090BB01A6016E2D8F2D0A
:1038E0000E943707D0E08111EACF8E0183E0000FFC
:1038F000111F8A95E1F7F801E054FE4F81818E1186
:10390000DECF80818F11DBCF82818111D8CFE38020
:10391000F480EC18FD0860E087EB91E00E946010F5
:103920008091670390916803E816F90640F680914C
:10393000BC018F7080618093BC01F801EB53FE4F96
:1039400080818F708061808387EB91E00E94731586
:10395000DF91CF911F910F91FF90EF90DF90CF906B
:103960000C943F0A3F924F925F926F927F928F9298
:103970009F92AF92BF92CF92DF92EF92FF920F93FE
:103980001F93CF93DF93CDB7DEB765970FB6F8944B
:10399000DEBF0FBECDBF8C0185E0F801DE01519680
:1039A00001900D928A95E1F7D8014C9011965C90A8
:1039B00011971296EC9012971396CD90DC9060E0E0
:1039C00087EB91E00E94601087EBA82E81E0B82E73
:1039D0008090BA019090BB01A4016091B8018091E0
:1039E000B7010E9437078111CAC1F090B901F601F1
:1039F000E819F9094F0160E0FF2009F46DC1C50124
:103A00000E94601060906703709068033090BC0162
:103A10008614970408F013C14091BA015091BB017C
:103A2000B090B701A090B801832D807F6A2D09F076
:103A3000ADC08B2D0E943707FE2C81113BC0D801F1
:103A400011968C9111978A1135C08C918B1132C0CF
:103A50002091BD013091BE0116968D919C91281741
:103A6000390741F5E11026C0832D8F708061809366
:103A7000BC0187EB91E00E9473158091BC01F801B5
:103A800085838F2D65960FB6F894DEBF0FBECDBF30
:103A9000DF91CF911F910F91FF90EF90DF90CF902A
:103AA000BF90AF909F908F907F906F905F904F905E
:103AB0003F900895F4EF6F16F1E07F0620F48091B7
:103AC0006C0380FF21C0A601652D842D0E9437075D
:103AD000811118C081E08E2580FF16C04E2D652D06
:103AE000842D0E941F0A882379F087EB91E00E94C1
:103AF000731588E0E7EBF1E0DF011D928A95E9F7A5
:103B0000F12CBFCF80E0E8CFA601652D842D0E9467
:103B10003707811124C081E08E25B82FB170CB2EDC
:103B200080FF2BC04E2D652D842D0E941F0AD82E9C
:103B3000811123C0498A5A8A89899A890E941D1055
:103B4000292F22952F70223060F0243088F49F7046
:103B500061F0F8019581907F41F4FD2C92CF80E0D7
:103B6000DCCF9F7011F08823C1F3805E8830A8F30A
:103B7000C8010E947315DC2CF0CFEE2009F481CF30
:103B80008091BC0181608093BC01BACF8B2D0E94D3
:103B90003707811124C0D80111968C9111978A1191
:103BA0001EC08C918B111BC02091BD013091BE01B4
:103BB00016968D919C9117972817390781F4E1107B
:103BC0000EC015963C92C8010E94731588E0F8015A
:103BD000A7EBB1E001900D928A95E1F752CFC801B1
:103BE0000E942910882339F1EE2029F18091BC012F
:103BF0008032A0F02091B7013091B8013A8729872F
:103C00001B86DD86CC868E878091BD019091BE019A
:103C1000988B8F87CE0109960E94731588E0F80172
:103C2000A7EBB1E001900D928A95E1F70E94441C48
:103C3000FF24F39426CFC8010E947315F9CF832D7A
:103C4000807F09F452CF9090B7018090B8014091E5
:103C5000BA015091BB01682D892D0E94370781114F
:103C60001CC0F8018181881118C08081891115C09C
:103C70002091BD013091BE018681978128173907B7
:103C800061F4E1100AC03582C8010E94731588E012
:103C9000D5011D928A95E9F7F4CEC8010E9429103A
:103CA000882349F2EE2039F28091BC01803208F479
:103CB000B5CF2091B7013091B8013A8329831B8297
:103CC000DD82CC828E838091BD019091BE01988768
:103CD0008F83CE010196A0CF87EB91E00E94601008
:103CE00080916703909168038816990680F6FE2CF0
:103CF000EE2009F4A0CFE090B701D090B801409138
:103D0000BA015091BB016D2D8E2D0E943707811194
:103D100028C0F80181818D1124C080818E1121C0BD
:103D20002091BD013091BE01868197812817390706
:103D3000C1F480916C0382FD49CF9091BC0190FD4C
:103D400045CF907F09F442CF8091BC018583903F9D
:103D500009F439CF982F907F905F8F70892B8583DE
:103D600032CFC8010E942910811158CF8091BC0127
:103D700081608093BC01C8010E94731582CEEE2041
:103D800009F459CFC8010E942910F82E882309F49C
:103D900052CF88E0F801A7EBB1E001900D928A952F
:103DA000E1F78091B7019091B8010E941D100E9427
:103DB000441C67CECF93DF93CDB7DEB760970FB6C5
:103DC000F894DEBF0FBECDBF29873A874B875C874B
:103DD0006D877E878F87988BCE0109960E94B21CD3
:103DE00081112FC088E0FE013996DE011196019005
:103DF0000D928A95E1F74C855D856A8589850E94DB
:103E0000370781111EC0A091BF01B0E0CD0101961E
:103E100087709927209100022817190609F193E06D
:103E2000AA0FBB1F9A95E1F7A054BE4F98E0FE0180
:103E3000319601900D929A95E1F78093BF010E940F
:103E40003F0A809100029091BF01891317C06096CC
:103E50000FB6F894DEBF0FBECDBFDF91CF910895AE
:103E60000E94D1111092BF011092000288E0E7EB8E
:103E7000F1E0DF011D928A95E9F7E3CFB8E08B9F6F
:103E8000C001112480549E4F0E94B21C8823F9F275
:103E90008091000290E0019687709927809300023C
:103EA000D0CFEF92FF920F931F93CF93DF93809128
:103EB000AA02882361F0C091A9028CE0F82E8091BB
:103EC000AA02C81758F01092AA021092A902DF9114
:103ED000CF911F910F91FF90EF900895EE24E394FE
:103EE000EC0EE092A9020C2F10E0CF9DE00111240E
:103EF000C555DD4F4B815C81698188810E94370700
:103F000081111BC08E819F81892B21F48885998521
:103F1000019651F4288139814A815B816C817D81D0
:103F20008E819F810E94DA1EF09EF001F19EF00DBD
:103F30001124E555FD4F14821382CE2DC0CF10926F
:103F40004E0310924D031092130180914C03809305
:103F50004B030E9470070C94511F3F924F925F9247
:103F60006F927F928F929F92AF92BF92CF92DF9289
:103F7000EF92FF920F931F93CF93DF93C0914B0368
:103F800097E0892E01E010E02CE0322E3EEF932ED8
:103F90004424439480914C038C1315C00E94511FFC
:103FA000DF91CF911F910F91FF90EF90DF90CF9015
:103FB000BF90AF909F908F907F906F905F904F9049
:103FC0003F900C947007D0E0FE01EE0FFF1FED5BF9
:103FD000FC4F80819181889ED001899EB00D112473
:103FE000A55FBC4F14962C911497211157C0509087
:103FF000AA02EBEAF2E030E020E0712C5D01251529
:1040000008F04AC0E284F384D501CD90DC906FEFD4
:104010007FEF612C462D50E0DA01AA0FBB1FAC0DDB
:10402000BD1D0D90BC91A02D109731F0EA16FB0636
:1040300009F4BA016394EECF6F3F7607A1F1D8017E
:1040400002C0AA0FBB1F6A95E2F77A2AB80102C024
:10405000660F771F6A94E2F7AB014150510974165D
:104060001506F9F4329EF001339EF00D1124E5554A
:10407000FD4F889ED001899EB00D1124A55FBC4FD5
:1040800012962D913C9113973783268390829182CB
:104090009187808715964C920E9442072196C370A3
:1040A00079CF148213822F5F3F4F3C96A8CF2F9277
:1040B0003F924F925F926F927F928F929F92AF92B8
:1040C000BF92CF92DF92EF92FF920F931F93CF9305
:1040D000DF93CDB7DEB769970FB6F894DEBF0FBE9A
:1040E000CDBF942F498B252F5A8B6B8B7C8B8D8B5F
:1040F0004C895D89622F892F0E943707811109C081
:10410000809185019091860101969093860180931C
:1041100085018B89811110929A031D861E861F8648
:10412000188A85E0FE017196DE01199601900D92C4
:104130008A95E1F780910B0282FD1EC080915103A8
:1041400090915203892BC1F00E94F3062091020244
:1041500030910302821B930B209151033091520343
:104160008217930720F08091040282FFF5C10E941C
:104170007F0981110E944C094C855D856A8589857E
:104180000E943707811111C061E0CE0109960E949B
:1041900060106C018B8527EFC2162CE5D20681F4E6
:1041A000882321F181E08093130129853A854B858D
:1041B0005C856D857E858F8598890E94DA1EC5C0D5
:1041C00038EFC3163CE5D30629F4882379F00E9422
:1041D0009F1FEBCF49EFC4164CE5D40639F4882372
:1041E00029F0809113018111F2CFDCCF0BE013E0B5
:1041F000512CB12CA12C22242394312C2EEF422EB1
:10420000F8014081518188248A94982C20E0822FE3
:1042100090E0FC01EE0FFF1FE40FF51F608171813C
:104220006115710531F0C616D70609F44C012F5FF0
:10423000EECFF12CFFEF8F169F0609F448C0F8016E
:104240004481F09013018F2D411180E0F82FF1701F
:10425000FF2EF801E58086819B85992309F40CC126
:10426000FF2009F409C16090650370906603E110B6
:1042700012C0A10101C0440F8A94EAF7842B8683FF
:104280008091A7029091A8028615970520F470925C
:10429000A8026092A702C10102C0880F991F2A9547
:1042A000E2F70197F80126812817190681F4809119
:1042B0004D0390914E03009709F460C00E94E406FC
:1042C0006816790608F05AC021E0F80124835F28B7
:1042D000FFEFAF1ABF0A095F1F4F28E0A216B10413
:1042E00009F08ECF8B85882309F421C1552009F46C
:1042F0001EC10E94F30690934E0380934D0380915C
:10430000AA02883010F591E0980F9093AA0298E0E5
:10431000FE013996DE01119601900D929A95E1F712
:104320003CE0839FC001112485559D4F28E0FE018C
:104330003196DC0101900D922A95E1F72FEF3FEFC6
:10434000FC0131872087D386C28669960FB6F89420
:10435000DEBF0FBECDBFDF91CF911F910F91FF90B8
:10436000EF90DF90CF90BF90AF909F908F907F9015
:104370006F905F904F903F902F90089580914B03E6
:1043800050914C03982FF0E0E0E0851314C0909317
:104390004B03E017F10709F49ACF90E0FC01EE0F10
:1043A000FF1FED5BFC4FB182A082019683709927BD
:1043B00080934C038CCF682E712CF301EE0FFF1FFE
:1043C000ED5BFC4F2081318147E0429FD001439F4C
:1043D000B00D1124A55FBC4F6D917C911197798F21
:1043E000688F40E020E030E0E32FF0E0EE0FFF1FA9
:1043F000688D798DE60FF71F80809180811491047C
:10440000E1F0F8010190F081E02DFF8BEE8B20E0D0
:1044100005C08616970609F44F2D2F5FE22FF0E0B6
:10442000EE0FFF1F6E897F89E60FF71F6081718194
:104430006115710571F73F5FD7CF4423D1F0F801C3
:10444000231708F0FD0121E024830E171F0721F434
:1044500090934B03F42E3BCF981305C0AE17BF07C4
:1044600011F49F5F937093012F5F3F4F822F8370F2
:104470008CCFF0E0E0E0F7CF90E0E1101FC0B10199
:1044800002C0660F771F2A95E2F79B012150310980
:104490008217930731F4442309F447C0C5010E94F1
:1044A0004207C10101C0880F8A94EAF7982F9095BE
:1044B000F801868189238683FE2C09CF9C01082C74
:1044C00002C0359527950A94E2F7A9014170552756
:1044D000BC016150710986239723892B11F5452B67
:1044E00001F1F80182819381892BC1F01B821C822A
:1044F0001D821E8249824A820E94F3068160582FE3
:104500009D838C83F801828193818F839887298191
:104510003A814B816D817E810E94DA1EF8011582FD
:10452000C0CFF22FF170EF2EBCCFEF2CBACF90910D
:104530004B0380914C03981731F00E94AD1F55201A
:1045400009F433CE02CF0E94511F10924E031092F5
:104550004D030E947007F3CF82E00E94EE0A07CE5F
:10456000589850982FEF87EA91E62150804090406C
:10457000E1F700C00000ECE0F2E0119222E0EC3143
:10458000F207D9F790E080E00E94372A8A3E9E4FDA
:1045900021F40E946E10811102C00E94091582E070
:1045A00090E00E942F2A80931D020E948710909312
:1045B0000B0280930A020E94FA228FEF96E721E015
:1045C000815090402040E1F700C000000E94FA2294
:1045D00080910C0280FF08C06FEF7FEF90E080E0D9
:1045E0000E945B2A0E94D30683E090E00E942F2A5B
:1045F0000C942B0BEF92FF920F931F93CF93DF93AB
:10460000CDB7DEB728970FB6F894DEBF0FBECDBF8B
:1046100000910001109101018FEF9FEF9093010134
:10462000809300010F3F100709F088C080917A0144
:1046300090917B010E94E4060C9778F4F12C8F2D69
:1046400028960FB6F894DEBF0FBECDBFDF91CF9195
:104650001F910F91FF90EF9008950E94F3069093A1
:104660007B0180937A0119821A821B821C821D822F
:104670001E821F821886F894509A83EF9BE0019760
:10468000F1F700C000000E941F0F8CE20E94390F5A
:104690000E942C0F84EF91E00E940D0F892B11F4E2
:1046A0007894CCCF84EF91E00E94160F892BC1F350
:1046B00088E290E00E940D0F892B91F384E690E050
:1046C0000E94160F10E0892B59F382E890E00E94B7
:1046D0000D0F882339F17C01FF24C7010E94160FBA
:1046E000882301F11034C0F4E12FE695E695E695B4
:1046F00021E030E02C0F3D1F2E0F311DF90190817C
:10470000990F22E830E02E193F09E81AF1082E151A
:104710003F050CF450C0908381E0810F1F3F09F0EA
:1047200048C010E07894169516951695123009F049
:1047300085CF09811A81102701271027011511053E
:1047400009F47CCF8FE70F37100721F00F3F1007D8
:10475000A1F58FEF0E94EA0B809113018823F9F0F5
:1047600080914D0390914E030097C9F00E94E4069A
:104770002091A7023091A8022817390780F4909160
:104780004B0380914C03981761F10E94AD1F10926A
:10479000A8021092A70210924E0310924D0380912E
:1047A0006A03282F2170F22E80FD24C0FF24F39489
:1047B00046CF182F8ACF9160AECFF02E1F3F19F44D
:1047C0000E94B0223CCF812F0E94EA0B9FEF091775
:1047D00019F2102F00270F6F1093010100930001B1
:1047E000BBCF0E94511F10924E0310924D030E94A6
:1047F0007007D5CF8091120182FFD8CF0E94F306B7
:104800002091A3023091A402AC01421B530B2091D2
:104810001001309111014217530740F22CE731E0AB
:1048200041E0BC018091A5029091A6020E94210D59
:1048300006CF1F920F920FB60F9211242F933F9322
:104840004F935F936F937F938F939F93AF93BF9398
:10485000CF93DF93EF93FF93D091E900DF708091C6
:10486000EC00C82FC17080FDC0E81092E900809173
:10487000F000877F8093F00078940E94DC11109202
:10488000E9008091F00088608093F000CD2BCF701C
:10489000C093E900FF91EF91DF91CF91BF91AF916C
:1048A0009F918F917F916F915F914F913F912F9148
:1048B0000F900FBE0F901F9018951F920F920FB67A
:1048C0000F9211242F933F934F935F936F937F9396
:1048D0008F939F93AF93BF93EF93FF938091E100EA
:1048E00082FF09C08091E20082FF05C08091E10053
:1048F0008B7F8093E1008091DA0080FF24C080915B
:10490000D80080FF20C08091DA008E7F8093DA008B
:104910008091D90080FF9DC080E189BD82E189BD81
:1049200009B400FEFDCF81E080938F038091820364
:10493000811109C00E9444050E940F068091E20087
:1049400084608093E2008091E10080FF17C0809135
:10495000E20080FF13C08091E2008E7F8093E2002E
:104960008091E20080618093E2008091D8008062B3
:104970008093D80019BC85E080938F038091E1007B
:1049800084FF2BC08091E20084FF27C080E189BDB5
:1049900082E189BD89B5982F917080FFFBCF80910E
:1049A000D8008F7D8093D8008091E1008F7E809326
:1049B000E1008091E2008F7E8093E2008091E2002E
:1049C00081608093E20080919003882309F447C0BE
:1049D00084E080938F0380918F038091E10083FFB7
:1049E00027C08091E20083FF23C08091E100877F90
:1049F0008093E10082E080938F0310929003809176
:104A0000E1008E7F8093E1008091E2008E7F8093B1
:104A1000E2008091E20080618093E20042E060E089
:104A200080E00E94DD058091F00088608093F000B6
:104A3000FF91EF91BF91AF919F918F917F916F9176
:104A40005F914F913F912F910F900FBE0F901F904C
:104A5000189519BC10928F031092820374CF809125
:104A6000E30087FD93E090938F03B5CF78941F9276
:104A70001FB61F9211248F939F93AF93BF93809182
:104A80007B0390917C03A0917D03B0917E030196FE
:104A9000A11DB11D80937B0390937C03A0937D03A4
:104AA000B0937E03BF91AF919F918F911F901FBED6
:104AB0001F9018951F921FB61F9211248F939F93DA
:104AC000AF93BF9380917A03811113C080917B03D0
:104AD00090917C03A0917D03B0917E034196A11D2E
:104AE000B11D80937B0390937C03A0937D03B093CF
:104AF0007E03BF91AF919F918F911F901FBE1F901A
:104B00001895CDB7DEB7E4970FB6F894DEBF0FBEA9
:104B1000CDBF84B7877F84BF0FB6F894A8958091E6
:104B20006000886180936000109260000FBE80E892
:104B300090E00FB6F89480936100909361000FBEEF
:104B400085B7806885BF85B7806885BF8AE897E0AC
:104B500090937101809370010E94B0140E94860F9F
:104B60000E9444050E940F068091E20084608093B9
:104B7000E200789480918F038823A1F01091E900DE
:104B80001F709091EC00892F817090FD80E8182BA8
:104B90001092E9008091E80083FD0E94DC111F70F3
:104BA0001093E90082E084BD93E095BD9AEF97BD34
:104BB00080936E000E946E10811102C00E94C2118B
:104BC0000E94B02282E091E0909377038093760375
:104BD00038E1432E512C40E4342ECE0101965C0185
:104BE0007E0191E2E90EF11C54E1652E59E0752E2B
:104BF00080918F0300E112E1853009F4BCC00E946E
:104C0000FA22882359F08FB7F89440917B03509192
:104C10007C0360917D0370917E038FBFACE0B2E0B6
:104C2000EEE1F2E010E000E0302F8D9191919817C5
:104C300009F4B3C0292F282790E0DD24D394422F14
:104C40004D2109F4A5C09BA73CA78D2191E009F453
:104C500090E09DA70E94F3068160782F9FA78EA702
:104C60004BA55CA56DA58FA50E945720F801E25EBB
:104C7000FD4F8081D826D0820E942B0790911C0284
:104C8000891739F00E942B0780931C0280950E949F
:104C9000610F80918F03843009F0AACF83E0809365
:104CA000E9008091E80082FFA3CF8091E80090E0C6
:104CB00085FF06C00E946305882309F485C091E042
:104CC0008091E8008B778093E800992309F490CFD6
:104CD000009180021091810289810115110509F46A
:104CE0008FC08E3F09F0D7C08A81833020F0855075
:104CF000833008F0D0C0EA81EE3008F0CCC0F0E09C
:104D0000E156F54D0C94F92980918F03843021F1FF
:104D10008FEF0E94610F10927A030FB6F894A89556
:104D2000409260000FBE3092600083B7817F846044
:104D300083BF83B7816083BF7894889583B78E7F64
:104D400083BF0FB6F894A895809160008861809326
:104D50006000109260000FBE80918E03882359F08E
:104D60000E94FA22ECE0F2E081918111A4C222E0DB
:104D7000EC31F207C9F780918F03853009F4C4CF75
:104D80000E94D1110E942B0780950E94610F37CF9E
:104D90009F5FDD0C983009F052CF0F5F1F4F00313D
:104DA000110509F041CF8FEF88AB89AB1AAA0E9499
:104DB000F3068160782F9CAB8BAB48A959A96AA9EF
:104DC0008CA90E94572058CF00E210E0CE01019636
:104DD0006C018091E80085FD0AC08091E8008B7726
:104DE0008093E8000E946305882399F368CF80913F
:104DF000F100F60181936F010150110951F75FCF66
:104E00008D3009F496C0B0F4843009F479C040F4D0
:104E1000823041F108F065C0813001F18FEF77C237
:104E2000863009F483C008F476C08C30B9F780E18D
:104E30008A8331C0813109F4D4C040F48F3009F441
:104E4000A4C008F479C00E94D51025C0833109F4AC
:104E5000F2C008F4C8C08E3F09F74DCF1A8289E02E
:104E60008B8319C08A81823009F473C2833099F030
:104E70008130A1F62FB7F89460917B0370917C0389
:104E800080917D0390917E032FBF0E94FF296B8349
:104E90007C838D839E8380918F03843009F0A8CE1C
:104EA0001091E9001F709091EC00892F817090FDA6
:104EB00080E8182B82E08093E9008091E80080FF71
:104EC0000CC050E040E060E270E0C5010E94940533
:104ED0008091E8008E778093E8001F701093E900BE
:104EE00087CE8A81823009F099CF6B817C818D8158
:104EF0009E810E94FF2986E290E00E943D2ACBCF4E
:104F00004C816B818A810E94AC0F98278927982752
:104F10009E838D83C0CF2D813E8132272327322768
:104F20004C816B818A810E94E510B5CF0E944F11A0
:104F3000B2CF1A8287E694CF0C8110E00D311105B3
:104F400008F0A9CF8A809B80982489249824CE01D8
:104F500001966C01080F191FC40187569C4FC0169B
:104F6000D10609F498CFE7E68E16910458F40E9412
:104F70002F2AF6018483FFEF8F1A9F0A2FEFC21AA0
:104F8000D20AEACFF6011482F6CF80910E019091F9
:104F90000F01892B09F47FCFCC80D12C4DE1C416B1
:104FA000D10408F078CF0A811B8110270127102730
:104FB000CE0101964C01C00ED11EC80187569C4FF0
:104FC000C016D10609F467CF0736110520F4F401A5
:104FD00064810E943D2AFFEF8F1A9F0A0F5F1F4FC7
:104FE000ECCF83E025CF0C8110E00D31110508F0E6
:104FF00052CF8A809B80982489249824CE010196E0
:105000006C01080F191FC4018796C016D10609F458
:1050100042CF8114E3E09E0658F40E942F2AF60145
:105020008483FFEF8F1A9F0A2FEFC21AD20AEBCFA9
:10503000F6011482F6CFCC80D12C4DE1C416D104F8
:1050400008F029CF0A811B8110270127102701159D
:1050500083E0180708F01FCF80E093E0801B910BDE
:105060008C159D0508F417CFFE0131964F01C00E37
:10507000D11EC8018796C016D10609F40CCF0115C0
:10508000F3E01F0720F4F40164810E943D2AFFEF42
:105090008F1A9F0A0F5F1F4FECCF88E0E5E1F1E028
:1050A000D70101900D928A95E1F780E2F501119206
:1050B0008A95E9F784E0898388E0F701DE01159697
:1050C00001900D928A95E1F7E6CE84ED898383E025
:1050D0008A831B821C82DFCE8C81682F70E0762F42
:1050E00066278B81860F972F911D092E000CAA0B26
:1050F000BB0B25E0880F991FAA1FBB1F2A95D1F76C
:10510000AC01BD01405E5F4F6F4F7F4F481759079D
:105110006A077B0708F4BFCE843DF3E09F07A10533
:10512000B10508F0B8CE453D23E052076105710591
:1051300020F044ED53E060E070E0481B590BBC01E7
:1051400060517E4FC5010E94062AA5CE4EE150E077
:105150006FEF70E0CE0103960E94182A80910E0135
:1051600089830A8398CE81E090E0909381028093B6
:10517000800282E390E090932F0280932E020E949F
:10518000F30689CE80910E0189830A8380912E02D5
:1051900067CE0B811C8140E250E06FEF70E0C501EB
:1051A0000E94182A24EC38E090E080E0AC014E5FC9
:1051B0005F4F4132510508F06ECEF901659174914F
:1051C0000617170730F48A0D9B1DFC01718360835D
:1051D000CA01285F3F4F6216730641F75CCE2B81F0
:1051E0003C8184EC98E0FC014591549142175307AF
:1051F00009F477C00896F9E084319F07A1F70ECE35
:105200008B819C8104EC18E0F80125913491821780
:10521000930709F47EC0085F1F4F29E0043112078D
:1052200099F7FCCD0E94B21036CE8B81833059F0B5
:10523000843029F181112FCE80E2F50111928A95F7
:10524000E9F788E0F5CD6C818AE0F701282F11920B
:105250002A95E9F7683088F4689FB0011124675BEC
:105260007C4F4AE050E0C7010E941F2A80E08983FA
:105270008AE0F701DE01129623CF8FEFF8CF6C8121
:105280008AE0FE013596D70101900D928A95E1F7EB
:105290008FEF683060F44AE0649FB0011124675BCF
:1052A0007C4F4AE050E0C7010E94612A80E0898378
:1052B0000E94B014F0CD09BD19BD09B400FEFDCFA8
:1052C0008091D8008F7D8093D8008091E00082602B
:1052D0008093E0008091E00081FDFCCF0E94D1111D
:1052E0004ACD9C012E5F3F4FF901459154914032C8
:1052F000510508F093CDF90145915491FC01349684
:1053000065917491CE0102960E940F2A80E08983F4
:10531000C2CDC8010296FC01259134912D31310591
:1053200008F07CCDFC0145915491F80134968591AB
:105330009491BE016B5F7F4F0E940F2A0E949510CF
:10534000F801369685919491009701F3FC01099537
:10535000DDCF86E290E00E942F2A1B821C821D82F4
:105360008E8399CD089590E080E008958FEF9FEFB0
:105370000895862F0E948A0781E090E00895EBE966
:10538000F3E01382128288EE93E0A0E0B0E0848321
:105390009583A683B78381E691E091838083089506
:1053A000CF92DF92EF92FF920F931F93CF93DF93F1
:1053B0006C017B01E40EF51E10E000E06E157F0528
:1053C00071F0EB01D601ED91FC910190F081E02D9F
:1053D0006991C6010995080F191FBE01EFCFC801D9
:1053E000DF91CF911F910F91FF90EF90DF90CF90C1
:1053F0000895EE0FFF1F0590F491E02D09946927A1
:10540000962769277827872778270895FB01DC01ED
:1054100002C005900D9241505040D8F70895FB010D
:10542000DC0102C001900D9241505040D8F7089520
:10543000DC0101C06D9341505040E0F70895DC015C
:10544000CB01FC01F999FECF06C0F2BDE1BDF89A8F
:10545000319600B40D9241505040B8F70895F99933
:10546000FECF92BD81BDF89A992780B50895A8E135
:10547000B0E042E050E00C94212A262FF999FECFAB
:1054800092BD81BDF89A019700B4021639F01FBA97
:1054900020BD0FB6F894FA9AF99A0FBE08950396B4
:1054A000272F0E943E2A0E943D2A252F0E943E2A35
:1054B000242F0C943E2A0196272F0E943E2A0C94FA
:1054C0003D2ADC01CB0103C02D910E946C2A415082
:1054D0005040D0F70895262FF999FECF1FBA92BDFC
:1054E00081BD20BD0FB6F894FA9AF99A0FBE0196C5
:1054F0000895F894FFCFB10AB10ABA0ABA0ABC0AF1
:10550000BA0ABA0ABA0AB10AB10AC10ABA0ABA0A86
:10551000C10AC212EA129814EA1298141D133E131B
:1055200098144714541448194819811981194D1AAF
:10553000BA19BA19BA19691AD61AE71AE71A4D2808
:1055400065286C284B274B27A628B328C2284B2751
:0A555000C928EF28002912291529A7
:10555A00FFFFD006350CCF06310C2D0CCE0601000C
:10556A00AF00010101EC1A0C495526606081828363
:10557A00E200E900EA00B500B600B700CD008301F9
:10558A00CC008A01920194012102230224022502FD
:10559A00260227022A02B300B4006F0070004022DC
:1055AA00320001DE00AC0026093F095F0900000055
:1055BA0000B929D029B329B629B629B229B22900B6
:00000001FF
